:030000000248C7EC
:0C48C70078FFE4F6D8FD75816C02490E04
:101873000A53746172743A20004950436F6E6E6567
:1018830063745245510A004950436F6E6E65637429
:10189300003E432C562C43432CC0E4E0EFF2E5F02A
:1018A30020D1E8EDEAEEEC49500A003E432C4D41CD
:1018B300432C25303262583A25303262583A25306B
:1018C3003262583A25303262583A25303262583AF9
:1018D30025303262582C4D414320E0E4F0E5F10A13
:1018E300003E432C5645522C20332E3020EEF2205E
:1018F30025732025732CC2E5F0F1E8FF2049502021
:10190300ECEEE4F3EBFF0A004F6374203033203234
:101913003030370031323A30313A3030003E432CE8
:101923004C442C50524F473A202020202020202086
:1019330020202020202020202020202020202020A4
:101943002020202020202020202020202020202094
:101953002020202020202020202020202020202084
:10196300202020202020202020202020202CC4E004
:10197300F2E020EFF0EEF8E8E2EAE828F4E0E9EB41
:10198300290A003E2A2C312CCEF1EDEEE2EDFBE5E7
:1019930020EFE0F0E0ECE5F2F0FB20F1E5F2E5E228
:1019A300EEE3EE20E8EDF2E5F0F4E5E9F1E00A001C
:1019B3003E412C4130312C2562752E2562752E2532
:1019C30062752E2562752C495020E0E4F0E5F12084
:1019D300E0E4E0EFF2E5F0E00A003E412C41303272
:1019E3002C2562752E2562752E2562752E2562754E
:1019F3002C495020E0E4F0E5F120EEF1ED2E20F14A
:101A0300E5F0E2E5F0E00A003E412C4130332C25BD
:101A130062752E2562752E2562752E2562752C49F9
:101A23005020E0E4F0E5F120F0E5E72E20F1E5F0C9
:101A3300E2E5F0E00A003E412C4130342C2562758A
:101A43002E2562752E2562752E2562752CCCE0F14C
:101A5300EAE020F1E5F2E80A003E412C4130352C62
:101A63002562752E2562752E2562752E2562752CCD
:101A7300D8EBFEE70A003E532C4130362C25627525
:101A83002CC2F0E5ECFF20EEE6E8E42E20EAE2E8E3
:101A9300F2E0EDF6E8E820282A3130ECF1290A00DB
:101AA3003E2A2C312CC4EEEF2E20EFE0F0E0ECE5E3
:101AB300F2F0FB20F1E5F2E5E2EEE3EE20E8EDF2F1
:101AC300E5F0F4E5E9F1E00A003E422C5330312C15
:101AD3002562752CC6E4E0F2FC20E7E0EFF0EEF1BE
:101AE300E020F1EEE5E4E8EDE5EDE8FF20EEF2209D
:101AF300F1E5F0E2E5F0E00A003E422C5330322CEF
:101B03002562752C43E2FFE7FC20F120F1E5F0E2CA
:101B1300E5F0EEEC20EDE520EFEEE4E4E5F0E6E8B9
:101B2300E2E0F2FC0A003E422C5330332C2562756E
:101B33002CCFE5F0E5E7E0EFF3F1EA20EFF0E82062
:101B4300EFEEF2E5F0E520F1E2FFE7E820F120F126
:101B5300E5F0E2E5F0EEEC0A003E422C5330342C83
:101B63002562752CCDE5F220EFE5F0E5E4E0F7E83A
:101B730020E4E8E0E3EDEEF1F2E8EAE820E220F128
:101B8300E5F0E2E5F00A003E422C5330352C2562A5
:101B9300752CCAE0EDE0EB20F8E8F0EEEAEEE2E5C2
:101BA300F8E0F2E5EBFCEDEEE3EE20EEE1ECE5ED43
:101BB300E00A003E532C5330362C25303262582530
:101BC300303262582530326258253032625825301F
:101BD30032625825303262582C4D414320E0E4F004
:101BE300E5F120F8E8F0EEEAEEE2E5F8E0F2E5EB05
:101BF300FCEDEEE3EE20EEE1ECE5EDE00A003E4520
:101C03004E440A0044756D70582020202020303047
:101C13002030312030322030332030342030352012
:101C230030362030372030382030392030412030D2
:101C3300422030432030442030452030460A003AC9
:101C430020000A0044756D7044202020202030308D
:101C530020303120303220303320303420303520D2
:101C63003036203037203038203039203041203092
:101C7300422030432030442030452030460A00457E
:101C83007272206B657900526420656570726F6DA6
:101C93000A005264204D454D0A00526420436F648C
:101CA300650A0044656275674950204F4E0A004437
:101CB300656275674950204F46460A004465627560
:101CC3006755736572204F6E0A00446562756755E8
:101CD300736572204F46460A0044656275674D730B
:101CE30067204F6E0A0044656275674D7367204F26
:101CF30046460A00436F6E666967206C6F636B210B
:101D03000A00577220656570726F6D0A0020536177
:101D1300766520656570726F6D210A0045727220C9
:101D23004D414321004C6F61643E3E002A003C411B
:101D330030313D003C4130323D003C4130333D00C9
:101D43003C4130343D003C4130353D003C41303670
:101D53003D004E4F4950004C494E4B434F4E545259
:101D6300005452415353004652004E4F4C494E4B80
:101D730000494E49004E4F4449414700003C210071
:101D83003C5330313D003C5330323D003C53303303
:101D93003D003C5330343D003C5330353D003C5313
:101DA30030363D00FF1D55FF1D5AFF1D64FF1D6AA0
:0C1DB300FF1D6DFF1D74FF1D78FF1D7FDC
:0652F500016900016700E1
:1052B100C2AFC28E758900438910758BFF758DB79A
:0752C100D2ABD28ED2AF2266
:03001B0002483167
:10483100C0E0C083C082C0D0C2AFC28E758BFF758D
:104841008DB720060675A61E75A6E10567D202E59D
:104851006960020569E568D3940140021568056C39
:10486100E56C540F704AD20DE56C543F7014D200C0
:10487100906F40E0600C04F0E0D394B44004C2AF08
:1048810080FE906F3BE0600204F09069B7E0600247
:1048910014F0906F41E0D394014003E014F030052F
:1048A10002056AE56BD394644004D2068002056B6D
:1048B100E566D3940140021566D28ED2AFD0D0D036
:0648C10082D083D0E0323A
:10125B00C291C290D2B5C20A7D027C007F071252A6
:10126B00458F26E526646060097D017F601251D9A8
:10127B00D20AE4FDFC7F0B1252458F26E52630E6A1
:10128B00097D04E4FF1251FDD20A7D017C007F072A
:10129B001252458F26E5267008FD7FFF1251D9D2D9
:1012AB000A300A03126000C2AFC288C2A8C2AA12D7
:1012BB004B5C906BF4E0B4FA09A3E064CE700302CC
:1012CB001352E4F52674EC2526F582E4346BF58392
:1012DB00E4F00526E526B443EC906BF474FAF0A326
:1012EB0074CEF0A374CCF0906BFA740AF0E4A3F014
:1012FB00A304F0A3F0906BFF7403F0A374CCF090F5
:10130B006BF074FFF0A3F0A3F0E4A3F0906C0B74FC
:10131B0005F0E4F526E5262401FFE433FE74EC2505
:10132B0026F582E4346BF583E0FD1252980526E531
:10133B0026C3944340DFE4F5A775A61E75A6E1907E
:10134B007FF0F0A3F080FED2AF906BFF7403F0A39D
:10135B0074CCF0E4906BFEF0124286EF6003123116
:10136B00DBC2B5122DD0C206124F99906C0BE0C3A5
:10137B00940350037403F0D20CD20BD20AD29320F5
:10138B000A077E187F7312436CE4906E2BF0125297
:10139B00B1C2AFA37408F0906B6A7424F0E4A3F0AD
:1013AB00906BF4E0906B6CF0906BF5E0906B6DF0E4
:1013BB00906BF6E0906B6EF0906BF7E0906B6FF0CC
:1013CB00906BF8E0906B70F0906BF9E0906B71F0B4
:1013DB00756801E4906E2DF0C207C208D2AF75A7F5
:1013EB000775A61E75A6E11251B3200A19AF267E0A
:1013FB00007D03124529E4FF1247877E6C7F2BE4A7
:10140B00FB7D01124603906F40E060037401F0E432
:10141B009069B7F0A37455F0A37481F0E4F56AE416
:10142B00F56B9069B7E070031224DA906F41E0B46A
:10143B0001119080007410F0E4906F41F0D20AD249
:10144B000BD20C908008E0F52630E405D20774101F
:10145B00F0E52630E508D2099080087420F0E526E7
:10146B0030E608D2089080087440F0E56AD3940304
:10147B004023908002E4F0908001F0908000F0E532
:10148B006AD39406400FE4F56AC203906E2DF07593
:10149B006801124F999080A0E07003124C55908018
:1014AB00B8E07003124CCF9080D0E07003124E174F
:1014BB00908000E07013300710124088906BE7EFBC
:1014CB00F0D394004003120A18908002E07006904B
:1014DB008000E06005D20502142AC205E4F56A908B
:1014EB0069B7E0600302142A300912123A6D906B4F
:1014FB00E7EFF0D394004005E0FF1252C820080339
:10150B000216891238F8906BE7EFF0700302142A79
:10151B00906C2BE054BF247F70030215EC14700306
:10152B000215C42402600302161F200A077E187FCF
:10153B007C12436C300E79200376906C03E07006BE
:10154B00906C07E0605B906F37E0FF906C03E0B549
:10155B000724906F38E0FE906C04E0B50618906F8E
:10156B0039E0FE906C05E0B5060C906F3AE0FE900A
:10157B006C06E06E602B906C07E06F7033906F38E9
:10158B00E0FF906C08E0B50727906F39E0FF906C97
:10159B0009E0B5071B906F3AE0FF906C0AE0B507C6
:1015AB000F906E2D7401F0120021756801021689DF
:1015BB00906F3774FFF0021689906F40E0600374F0
:1015CB0001F0906F2FE0FF906C2DE06F600302161F
:1015DB0089906F2FE004F0E4F568906E2BF0021603
:1015EB0089300303021689906BFAE0700302142A08
:1015FB001252FCD203E4F568906E2BF0906F3B0413
:10160B00F0E4906F2EF0A3F0200A737E187F8A12FD
:10161B00436C806A906F40E060037401F0300352BA
:10162B00906C2BE020E74B906C2DE0FF906F2EE041
:10163B00FE6F600D906F36E07007EE146F703F8099
:10164B0013906F2EE004F0906BE7E0FFD39404400F
:10165B00031250399068B37482F0A37401F0906C4C
:10166B002DE09068B5F07E687FB37D03124BDA02F4
:10167B00142A300E09200306906F3774FFF02003F5
:10168B000302173EE568706B125077EF60207E6D9A
:10169B007F2B906D2CE02404FD124BDA906F36E01B
:1016AB00600302142A906C0BE0F56802142A906F09
:1016BB003BE0D3943C403C906F36E07036906F3BF0
:1016CB0004F0906B69E0702B1252E2E4906D2BF0FA
:1016DB00A37412F0906F2FE0906D2DF0A374FDF0BA
:1016EB009069BA63A201906D2F63A2017F1212362B
:1016FB007D809B1252D7EF60159068B37483F0E432
:10170B00A3F07E687FB37D02124BDA02142AE568E0
:10171B006401600302142A906E2BE004F0E0C39482
:10172B00055003021699C203E4906E2DF0120021AE
:10173B0002142AE5686401600302142A906E2DE0FE
:10174B0014604024FE603C147003021826240460CD
:10175B000302142AE4F56A200E13906E2D7404F024
:10176B00906E2BE05401F075680102142AE4906E20
:10177B002DF0906E2B04F07568C8906F3774FFF0E6
:10178B0002142A906F37E07003021815906D2B74BA
:10179B0080F0906D2D7401F0E4A3F0A304F0A3741A
:1017AB0030F0A3747BF0E4F52674322526F582E441
:1017BB00346DF583747DF074332526F582E4346D36
:1017CB00F583E4F0E5262407906D2CF07C6F7D37D4
:1017DB00906BFFE0FAA3E0FB7F021249D87E6D7F8E
:1017EB002BE5262409FD124BDA906F36E0601B12B5
:1017FB0052FCD203E4F568906E2BF0906F3B04F033
:10180B00E4906F2EF0A3F002142A906E2D7404F066
:10181B00906C0BE02432F56802142A90800274104D
:10182B00F0756803906E2BE06401FFF0906E2D74E1
:10183B0001F0EF7019906C07E06013FCA3E0FDA3BF
:10184B00E0FEA3E0FF906F371229D202142A906CAE
:10185B0003E0FCA3E0FDA3E0FEA3E0FF906F3712D3
:07186B0029D202142A80FEBD
:011872002253
:100A1800906C2CE0B444047F0180027F00906C2B22
:100A2800E0B447047E0180027E00EE5F604A906B6E
:100A3800F4E0906C2DF0906BF5E0906C2EF0906BDC
:100A4800F6E0906C2FF0906BF7E0906C30F0906BC4
:100A5800F8E0906C31F0906BF9E0906C32F0906CAB
:100A68002C7452F0906B6363A2019080A863A2017A
:100A78007F0612367D021251906BE7E0C39408504E
:100A88000302125A906BF4E0FF906C2DE06F600344
:100A980002125A906BF5E0FF906C2EE06F60030233
:100AA800125A906BF6E0FF906C2FE06F6003021211
:100AB8005A906BF7E0FF906C30E06F600302125AB7
:100AC800906BF8E0FF906C31E06F600302125A906F
:100AD8006BF9E0FF906C32E06F600302125A906C81
:100AE8002CE0B44415906B63E0B4FF0E63A2019050
:100AF80080A863A2017F0612367D906F40E06003F4
:100B08007401F0906F417464F0906C2C7452F09002
:100B18006C2BE0646D6003020C957BFF7A18799466
:100B28001221E07BFF7A1879AE906BF4E0F52FA3E1
:100B3800E0F530A3E0F531A3E0F532A3E0F533A307
:100B4800E0F5341221E0752FFF75301975310B75FA
:100B580032FF7533197534177BFF7A1879E412213F
:100B6800E07BFF7A1979201221E07BFF7A197986D8
:100B78001221E07BFF7A1979B3906BFAE0F52FA385
:100B8800E0F530A3E0F531A3E0F5321221E07BFF78
:100B98007A1979DD906C03E0F52FA3E0F530A3E036
:100BA800F531A3E0F5321221E07BFF7A1A790B9038
:100BB8006C07E0F52FA3E0F530A3E0F531A3E0F5ED
:100BC800321221E07BFF7A1A7939906BF0E0F52F29
:100BD800A3E0F530A3E0F531A3E0F5321221E07B84
:100BE800FF7A1A795C906BECE0F52FA3E0F530A35F
:100BF800E0F531A3E0F5321221E07BFF7A1A79792A
:100C0800906C0BE0F52F1221E07BFF7A1A79A31282
:100C180021E07BFF7A1A79CCA20EE433F52F12215A
:100C2800E07BFF7A1A79FC906F36E0F52F1221E00D
:100C38007BFF7A1B7929906F40E0F52F1221E07B2A
:100C4800FF7A1B795C906B69E0F52F1221E07BFF3E
:100C58007A1B798AA201E433F52F1221E07BFF7A0F
:100C68001B79B6906F30E0F52FA3E0F530A3E0F5DF
:100C780031A3E0F532A3E0F533A3E0F5341221E027
:100C880012418C7BFF7A1C79011221E022906C2B97
:100C9800E0644C70527E1C7F0712436C906C33E00A
:100CA800F527A3E0F528E4F5297D03AF28AE271240
:100CB80045297E1C7F4212436CAE27AF28E4FB7D9A
:100CC800101246037E1C7F4512436C74102528F5CC
:100CD80028E43527F5270529E529C3941040CA7E5D
:100CE8001C7F4512436C22906C2BE0646C705CF5A1
:100CF8002B7E1C7F4712436CE4F52AAF2B7E007DC8
:100D0800031245297E1C7F4212436CE4F529A82B67
:100D1800E6FF74352529F582E4346CF583EFF00598
:100D28002B0529E529B410E67E6C7F35E4FB7D10A0
:100D38001246037E1C7F4512436C052AE52AC3949C
:100D48000840B87E1C7F4512436C22906C2BE064EF
:100D58004B7061F529741D2529F582E4346CF583FF
:100D6800E06032741D2529F582E4346CF583E0F4E3
:100D78006023741D2529F582E4346CF583E0FF7443
:100D8800332529F582E4346CF583E0B5071005298D
:100D9800E529B408C09069B77432F0021251906C1A
:100DA8002B7421F0300A030212517E1C7F821243F9
:100DB8006C021251906C2BE0B4521A200A077E1C68
:100DC8007F8A12436C906C2B7472F07E6C7F2B7D43
:100DD80008124A5C22906C2BE064497045200A078F
:100DE8007E1C7F9512436C906C33E0F527A3E0F5E9
:100DF80028E4F529852882852783E0FF743525298D
:100E0800F582E4346CF583EFF00528E528700205D7
:100E1800270529E529B480DC7E6C7F2B7D8A124A60
:100E28005C22906C2BE064437079A3E064527046B6
:100E3800200A077E1C7F9D12436C906C33E0F527D7
:100E4800A3E0F528E4F529852882852783E493FF24
:100E580074352529F582E4346CF583EFF00528E52F
:100E680028700205270529E529B480DB7E6C7F2BD5
:100E78007D8A124A5C22906C2CE06457600302124F
:100E88005A906C33E0F527A3E0F52874352529F549
:100E980082E4346CAD82FC7B80AF28AE27125126E9
:100EA800021251906C2BE064446003020F3C906C7A
:100EB80033E0FF64447003021251EFB4310CC20AEC
:100EC8007E1C7FA612436C021251906C33E0B43042
:100ED8000CD20A7E1C7FB212436C021251906C3302
:100EE800E0B4320CD20B7E1C7FBF12436C0212514D
:100EF800906C33E0B4330CC20B7E1C7FCD12436C74
:100F0800021251906C33E0B4340CD20C7E1C7FDC9E
:100F180012436C021251906C33E0B4350CC20C7E53
:100F28001C7FE912436C021251906C33E0FF1200EF
:100F38001E0212519069B7E07013200A077E1C7FC9
:100F4800F712436C906C2B7421F00212519069B720
:100F58007432F0906C2BE0FFB45104C2AF80FEEF06
:100F680064577045200A077E1D7F0512436C906CFC
:100F780034E0906BE7F0E4F529906BE7E0FFE529B2
:100F8800C39F400302125174352529F582E4346C5D
:100F9800F583E0FF906C33E025292462F582E43480
:100FA8006AF583EFF0052980D0906C2BE0645360DC
:100FB8000302105F200A077E1D7F1012436C906B9E
:100FC800F4E0FF906A6BE06F703C906BF5E0FF9087
:100FD8006A6CE06F7030906BF6E0FF906A6DE0B578
:100FE8000724906BF7E0FF906A6EE0B50718906BE6
:100FF800F8E0FF906A6FE0B5070C906BF9E0FF909E
:101008006A70E06F6016906C2B7421F0300A03024E
:1010180012517E1D7F1F12436C021251E4F529E420
:10102800F56BAF29FE74622529F582E4346AF583ED
:10103800E0FD1252980529E529C394FE40E1C2AFAC
:10104800E4907FF0F0A3F0907FFD74AAF0A374FF02
:10105800F0A37455F080FE906C2BE0644F704C90B8
:101068006C33E0F527A3E0F528E5284527700A202A
:101078000A077E1D7F2812436C200A077E1D7F2FDA
:1010880012436CE4F52974352529F582E4346CF5AE
:1010980083E0852882852783F00528E528700205E6
:1010A800270529E529B480DE021251906C2BE0FF58
:1010B800B44521906C33E0FDA3E0907FF0CDF0A320
:1010C800EDF0C2AF907FFD74AAF0A374FFF0A37493
:1010D80055F080FEEF64656003021251906C33E0B6
:1010E800FFA3E0907FF0CFF0A3EFF0E4F527F52819
:1010F800D3907FF1E09528907FF0E095274020E499
:10110800F56B2528FFE5273401FE8528828527838E
:10111800E0FD1252980528E5287002052780D17E47
:101128001D7F31124953EF4E6020120003906BFA75
:10113800EFF0120003906BFBEFF0120003906BFCD2
:10114800EFF0120003906BFDEFF07E1D7F37124920
:1011580053EF4E6020120003906C03EFF01200036F
:10116800906C04EFF0120003906C05EFF01200038E
:10117800906C06EFF07E1D7F3D124953EF4E6020C4
:10118800120003906C07EFF0120003906C08EFF068
:10119800120003906C09EFF0120003906C0AEFF054
:1011A8007E1D7F43124953EF4E6020120003906B5F
:1011B800F0EFF0120003906BF1EFF0120003906B68
:1011C800F2EFF0120003906BF3EFF07E1D7F4912EF
:1011D8004953EF4E6020120003906BECEFF01200C1
:1011E80003906BEDEFF0120003906BEEEFF012003E
:1011F80003906BEFEFF07E1D7F4F124953EF4E6067
:1012080008124F3C906C0BEFF0E4F529E4F56BE520
:10121800292401FFE433FE74EC2529F582E4346BBC
:10122800F583E0FD1252980529E529C3944340DC73
:10123800C2AFE4907FF0F0A3F0907FFD74AAF0A312
:1012480074FFF0A37455F080FE7E6C7F2B7D08122E
:021258004A5CEE
:01125A002271
:1050EE00AE07EEC39430400BEED394395005EE2448
:1050FE00D0FF22EEC39461400BEED394665005EEC2
:10510E0024A9FF22EEC39441400BEED394465005E2
:08511E00EE24C9FF22AF0622B6
:10527E00906B62E004F07006906B61E004F0906B4E
:0A528E0061E0FEA3E0FF125262226D
:1000030012527E1250EEEFC454F0FEC00612527E1E
:080013001250EED0E02FFF2295
:104F3C00E490706EF012527E90706FEFF0C394306C
:104F4C004018E0FFD39439501190706EE024BAF5FC
:104F5C0082E43469F583EFF0801190706EE024BA2E
:104F6C00F582E43469F583E4F0800C90706EE00413
:104F7C00F0E0D3940840BE752F00753000753100F9
:0C4F8C00E4F5327B017A6979BA123754DF
:014F980022F6
:044953008E2C8F2DEA
:10495700906B61E4F0A374FFF012527EEF606EF487
:10496700606B852D82852C83E493B507EC752E014A
:10497700E52D252EF582E4352CF583E4936025900B
:104987006B62E0252EFF906B61E03400FE125262ED
:10499700E52D252EF582E4352CF583E493B5070440
:1049A700052E80CCE52D252EF582E4352CF583E404
:1049B7009370A6E52E24FFFFE434FFFE906B62E0C0
:1049C7002FF0906B61E03EF07E007F0122E4FEFF56
:0149D70022BD
:104286007E1D7F80124953EF4E70037F01227E1DF3
:104296007F83124953EF4E600C12527EEF24D024D6
:1042A600FF920E8002D20E7E1D7F89124953EF4E79
:1042B600600C12527EEF24D0906F36F08005E490A9
:1042C6006F36F07E1D7F8F124953EF4E600C1252EF
:1042D6007EEF24D0906F40F08005E4906F40F07E32
:1042E6001D7F95124953EF4E600C12527EEF24D07B
:1042F600906B69F08005E4906B69F07E1D7F9B12E0
:104306004953EF4E600C12527EEF24D024FF9201E7
:104316008002C201906BF463A201906F3063A20128
:104326007F0612367D30013B7E1D7FA1124953EF79
:104336004E6030120003906F30EFF0120003906F62
:1043460031EFF0120003906F32EFF0120003906F1E
:1043560033EFF0120003906F34EFF0120003906F0A
:0643660035EFF07F00229C
:1031DB00C201E4906F40F0D20EC204906F36F090B3
:1031EB006B69F0906BF463A201906F3063A2017F67
:1031FB000612367DE4F527E52775F003A424A7F521
:10320B0082E4341DF583E493FB740193FA74029307
:10321B00F912280270030233CDE4F528F529FD7469
:10322B00E22DF582E43469F583E0FF70030233C8C5
:10323B00E52775F003A424A7F582E4341DF583E498
:10324B0093FB740193FA740293F9852882758300BA
:10325B0012281BFEEFB5060875290105280233C499
:10326B00E52970030233C4EE60030233BFE5272464
:10327B00FE60281470030233A71470030233AB14DF
:10328B0070030233B31470030233B72405600302D7
:10329B0033C8906F407401F00233C8D20174E22D31
:1032AB00F582E43469F583E0FF642D70030233C8C3
:1032BB001250EEEFC454F0FC74E32DF582E4346944
:1032CB00F583E0FF1250EEEF2C906F30F074E42D8D
:1032DB00F582E43469F583E0FF1250EEEFC454F04D
:1032EB00FC74E52DF582E43469F583E0FF1250EEB2
:1032FB00EF2C906F31F074E62DF582E43469F58391
:10330B00E0FF1250EEEFC454F0FC74E72DF582E4AD
:10331B003469F583E0FF1250EEEF2C906F32F074AE
:10332B00E82DF582E43469F583E0FF1250EEEFC42B
:10333B0054F0FC74E92DF582E43469F583E0FF1257
:10334B0050EEEF2C906F33F074EA2DF582E4346974
:10335B00F583E0FF1250EEEFC454F0FC74EB2DF547
:10336B0082E43469F583E0FF1250EEEF2C906F345A
:10337B00F074EC2DF582E43469F583E0FF1250EE26
:10338B00EFC454F0FC74ED2DF582E43469F583E061
:10339B00FF1250EEEF2C906F35F08021D204801D80
:1033AB00906F367401F08015C20E8011906B6974AA
:1033BB0001F08009E4F529F5280D02322A052702D0
:0233CB003202CC
:0133CD0022DD
:104FF200906E2CE0C3947C503D906E2CE0FE04F049
:10500200746A2EF582E4346BF583EFF0BF0A2790C1
:105012006E2CE0FF04F0746A2FF582E4346BF583A2
:10502200E4F0906E2CE0FF124ADE906E2C7408F0D1
:07503200906B6BE004F0221B
:104F99009080007480F0906BEC63A201F583F58238
:104FA90063A2017F0812367D906BF463A2019080A1
:104FB9008863A2017F0A12367D908092E4F0A3747F
:104FC90032F0A37401F0906BFEE0FF9080B1F09095
:104FD90080E1EFF09080957455F0A3F09080007413
:094FE90001F09080097470F022BF
:104C5500908009E04410F09080A0E0706C9080A1F5
:104C65007482F09080A874FFF0A3F0A3F0A3F07F06
:104C7500039080AEEFF07FCBA3EFF07F039080AC85
:104C8500EFF0A374CBF09080007402F09070601286
:104C950029DE00000000907060E0908040F0907088
:104CA50061E0908041F0907062E0908042F09070F9
:104CB50063E0908043F0A3E4F0A3F0A3F0A3F090A9
:094CC5008018F0A3F0A3F0A3F0A5
:014CCE0022C3
:104E1700908009E04440F09080D17482F0906BFF5D
:104E2700E0FF9080DEF0906C00E0FF9080DFF09074
:104E370080027402F09070641229DE000000009076
:104E47007064E0908058F0907065E0908059F09021
:104E57007066E090805AF0907067E090805BF0A3F6
:104E6700E4F0A3F0A3F0A3F0908030F0A3F0A3F058
:024E7700A3F0A6
:014E79002216
:104CCF00908009E04420F09080B8E0706C9080B93B
:104CDF007482F07F039080C6EFF07FCDA3EFF07F5B
:104CEF00039080C4EFF0A374CDF09080C074FFF0F8
:104CFF00A3F0A3F0A3F09080017402F090706812FB
:104D0F0029DE00000000907064E090804CF09070FD
:104D1F0065E090804DF0907066E090804EF090705E
:104D2F0067E090804FF0A3E4F0A3F0A3F0A3F0901E
:094D3F008024F0A3F0A3F0A3F01E
:014D48002248
:1049D8008C278D28A907EAFDE975F018A424ACFFF7
:1049E800E5F034808F82F583EDF0EBFDE975F01882
:1049F800A4FFAEF024ACFBEE34808B82F583A3EDEC
:104A0800F08528828C83E0FDEF24A8FFEE3480FE39
:104A18008F82F583EDF08528828C83A3E08F828EC8
:104A280083A3F0852882852783A3A3E0FDE975F099
:104A380018A424A8FFE5F03480FE8F82F583A3A391
:104A4800EDF08528828C83A3A3A3E08F828E83A3B5
:044A5800A3A3F02202
:064A5C008D2CAB07AA0639
:104A6200907060E0FCA3E0FDA3E0FEA3E0F5308ED1
:104A72002F8D2E8C2DAE02AF038E838F8263A20107
:104A8200E52F540744C0F58385308263A201AF2C21
:104A92001236E6908000E020E5F9E4FCFDFEE53008
:104AA200252CF530EE352FF52FED352EF52EEC3584
:104AB2002DF52D908040E52DF0A3E52EF0A3E52FF6
:104AC200F0A3E530F09080007420F0AF30AE2FAD4F
:0B4AD2002EAC2D9070601229D2AF2C8A
:014ADD0022B6
:064BDA008D27AB07AA06BF
:104BE000907064E0FCA3E0FDA3E0FEA3E0F52B8E53
:104BF0002A8D298C28AE02AF038E838F8263A20197
:104C0000E52A540744D0F583852B8263A201AF27A0
:104C10001236E6E4FCFDFEE52B2527F52BEE352AC2
:104C2000F52AED3529F529EC3528F528908058E549
:104C300028F0A3E529F0A3E52AF0A3E52BF0908066
:104C4000027420F0AF2BAE2AAD29AC28907064120C
:044C500029D2AF278F
:014C5400223D
:024787008F2879
:10478900908001E030E5037F0022907068E0FCA38F
:10479900E0FDA3E0FEA3E0F52C8E2B8D2A8C299059
:1047A9006F3063A201E52B540744C8F583852C8239
:1047B90063A2017F061236FCE52C2406F52CE435AC
:1047C9002BF52BE4352AF52AE43529F529906E2EA7
:1047D90063A201E52B540744C8F583852C8263A2A3
:1047E90001AF281236FCE4FCFDFEE52C2528F52C4A
:1047F900EE352BF52BED352AF52AEC3529F52990DF
:10480900804CE529F0A3E52AF0A3E52BF0A3E52CDC
:10481900F09080017420F0AF2CAE2BAD2AAC29901A
:0748290070681229D2AF28CC
:014830002265
:104088009081E0E0F527052705270527052705275F
:1040980005270527052705270527908010E0F52A1D
:1040A800A3E0F52BA3E0F52CA3E0F52D9081E1E04A
:1040B800F5270527052705270527052705270527A8
:1040C800052705270527908014E0F52EA3E0F52F96
:1040D800A3E0F530A3E0F531E530B52C08E531B5BE
:1040E8002D037F0022E4F527E530540744E0F583EB
:1040F80085318263A201906C2B63A2017F0812377D
:1041080014906C2D63A201906B6363A2017F061269
:10411800367D906C2BE0F528A3E0F529E4F527908F
:104128006C2BE0702AA3E024F8F527E53054074407
:10413800E0F58385318274082582F582E43583F5BC
:104148008363A201906C2B63A201AF27123714AED0
:1041580028E4FCFDE5312529F531E5303EF530ED63
:10416800352FF52FEC352EF52E908014E52EF0A383
:10417800E52FF0A3E530F0A3E531F090800074401E
:03418800F0AF276E
:01418B002211
:1038F8009081E6E0F52705270527052705270527F1
:1039080005270527052705270527908028E0F52A9C
:10391800A3E0F52BA3E0F52CA3E0F52D9081E7E0DB
:10392800F52705270527052705270527052705273F
:1039380005270527052790802CE0F52EA3E0F52F15
:10394800A3E0F530A3E0F531E4F527E530B52C0A1E
:10395800E531B52D05C208023A52E530540744F066
:10396800F58385318263A201906C2B63A2017F08E5
:10397800123714906C2BE0F528A3E0F529E52945CA
:103988002870099080027410F07F0022906F37E051
:10399800FFF4602D906C2DE06F7076906F38E0FF2B
:1039A800906C2EE06F706A906F39E0FF906C2FE09A
:1039B8006F705E906F3AE0FF906C30E06F6022802D
:1039C80050906C2DE0906F37F0906C2EE0906F382F
:1039D800F0906C2FE0906F39F0906C30E0906F3A77
:1039E800F0906C2BE0702AA3E024F8F527E530541A
:1039F8000744F0F58385318274082582F582E43521
:103A080083F58363A201906C2B63A201AF27123761
:103A180014AE28E4FCFDE5312529F531E5303EF505
:103A280030ED352FF52FEC352EF52EAF2DAE2CAD14
:103A38002BAC2AAB31AA30A92FA82ED31229A1402A
:103A4800099080027410F07F002290802CE52EF0FF
:103A5800A3E52FF0A3E530F0A3E531F090800274E0
:043A680040F0AF2754
:013A6C002237
:103A6D009081E3E0F527052705270527052705277D
:103A7D000527052705270527052790801CE0F52A32
:103A8D00A3E0F52BA3E0F52CA3E0F52D9081E4E068
:103A9D00F5270527052705270527052705270527C9
:103AAD00052705270527908020E0F52EA3E0F52FAB
:103ABD00A3E0F530A3E0F531E4F527E530B52C0AA8
:103ACD00E531B52D05C209023BB8E530540744E890
:103ADD00F58385318263A2019068B763A2017F0EE1
:103AED0012372A9068B7E0F528A3E0F5299068BF52
:103AFD00E0FFF46045906F30E0FEEF6E706EA3E076
:103B0D00FF9068C0E06F7064906F32E0FF9068C105
:103B1D00E06F7058906F33E0FF9068C2E06F704CAB
:103B2D00906F34E0FF9068C3E06F7040906F35E0A8
:103B3D00FF9068C4E06F60048032D28D9068B7E06A
:103B4D00702AA3E024F2F527E530540744E8F58305
:103B5D00853182740E2582F582E43583F58363A267
:103B6D00019068B763A201AF2712372AAE28E4FC93
:103B7D00FDE5312529F531E5303EF530ED352FF5F3
:103B8D002FEC352EF52EAF2DAE2CAD2BAC2AAB3147
:103B9D00AA30A92FA82ED31229A15006E529452810
:103BAD0070099080017410F07F0022908020E52E26
:103BBD00F0A3E52FF0A3E530F0A3E531F0908001FF
:053BCD007440F0AF2779
:013BD20022D0
:04436C008E2D8F2ED5
:10437000907060E0FCA3E0FDA3E0FEA3E0F5348EC6
:10438000338D328C31E534FFE5335407FEE42FF5ED
:1043900030EE34C0F52F853082F5837423F005307C
:1043A000E5307002052F532FC7F582852F83740ADD
:1043B000F00530E5307002052F532FC7906BF46382
:1043C000A201852F8385308263A2017F061236E623
:1043D00074062530F530E4352FF52F852D83852E95
:1043E0008263A201852F8385308263A2011236CABF
:1043F000908000E020E5F9E4FCFDFE907060E0F8BC
:10440000A3E0F9A3E0FAA3E02FFFEE3AFEED39FDB9
:10441000EC38FCEF2408FFE43EFEE43DFDE43CFC08
:104420009070601229D2907060E0908040F090709F
:1044300061E0908041F0907062E0908042F0907076
:0C44400063E0908043F09080007420F056
:01444C00224D
:064603008E2D8F2E8D2F7D
:10460900907060E0FCA3E0FDA3E0FEA3E0F5358E29
:10461900348D338C32E535FFE5345407FEE42FF54C
:1046290031EE34C0F530853182F5837423F00531DC
:10463900E531700205305330C7F582853083EBF0E0
:104649000531E531700205305330C7906BF463A230
:104659000185308385318263A2017F061236E674B3
:10466900062531F531E43530F530852D83852E82E7
:1046790063A20185308385318263A201AF2F12368F
:10468900E6908000E020E5F97408252FF52FFFE476
:10469900FCFDFEE5352FF535EE3534F534ED3533D2
:1046A900F533EC3532F532908040E532F0A3E5334D
:1046B900F0A3E534F0A3E535F09080007420F0AF65
:0D46C90035AE34AD33AC329070601229D2A2
:0146D60022C1
:024ADE008F4007
:104AE000907060E0FCA3E0FDA3E0FEA3E0F5448E3F
:104AF000438D428C41E544FFE5435407FEE42FFF1C
:104B0000EE34C0906B6A63A201F5838F8263A201C9
:104B1000AF401236E6908000E020E5F9E4FCFDFEAF
:104B2000E5442540F544EE3543F543ED3542F54285
:104B3000EC3541F541908040E541F0A3E542F0A31A
:104B4000E543F0A3E544F09080007420F0AF44AE5C
:0B4B500043AD42AC419070601229D2CE
:014B5B002237
:064529008E2C8F2DAB0566
:10452F00907060E0FCA3E0FDA3E0FEA3E0F5338E06
:10453F00328D318C30E533FFE5325407FEE42FF531
:10454F002FEE34C0F52E852F82F5837423F0052FBF
:10455F00E52F7002052E532EC7F582852E83EBF0C3
:10456F00052FE52F7002052E906BF463A201852EA7
:10457F0083852F8263A2017F061236E67406252FEC
:10458F00F52FE4352EF52E532EC7E52C852F82857A
:10459F002E83F0052FE52F7002052E532EC7F582BF
:1045AF00852E83E52DF0052FE52F7002052E532E56
:1045BF00C7908000E020E5F9E533240AF533E435B0
:1045CF0032F532E43531F531E43530F53090804055
:1045DF00E530F0A3E531F0A3E532F0A3E533F09039
:1045EF0080007420F0AF33AE32AD31AC30907060DC
:0345FF001229D2AC
:014602002295
:10526200E5D220E0FBC2AF438E2075D2028F828E40
:0B52720083E0FFE4F5D2538EDFD2AFE3
:01527D00220E
:10529800E5D220E0FBC2AF43D2028F828E83EDF0CD
:0952A80075D25063D250D2AF223E
:104B5C00E4FDED2401FFE433FE12526274EC2DF5FA
:104B6C0082E4346BF583EFF00DBD3FE6E4FDED24FC
:104B7C007FFFE433FE12526274E22DF582E4346955
:104B8C00F583EFF074E22DF582E43469F583E0707F
:104B9C001B74E22DF582E43469F5837420F074E320
:104BAC002DF582E43469F583E4F080040DBD80BEFC
:104BBC00E4906A61F0FDEDFF7E0012526274622D8A
:0D4BCC00F582E4346AF583EFF00DBDFEE9DB
:014BD90022B9
:025126008B2CD0
:10512800A2AF921EC2AF85A22D53A2FE8E838F829C
:1051380005A28C838D827409123742E52C53A2FE96
:1051480043A22012374453A2DF852DA2A21E92AF9C
:01515800FF57
:015159002233
:10524500A2AF921EC2AF8C838D82EF12374243A26A
:0C5255002012374453A2DFA21E92AFFFCC
:01526100222A
:0251D9008F271E
:1051DB00A2AF921EC2AFE4F5838D827406123742E2
:1051EB00E52743A22012374453A2DFA21E92AF7FC2
:0151FB0001B2
:0151FC002290
:0251FD008F27FA
:1051FF00A2AF921EC2AFE4F5838D82740A123742BA
:10520F00E52743A22012374453A2DFA21E92AF7F9D
:01521F00018D
:01522000226B
:1035A200A907E7FFA805EF93C3966008403B74FCA8
:1035B2002FFF80F00F08EF93C3966008402B74FB37
:1035C2002FFF80E00F08EF93C3966008401B74FA48
:1035D2002FFF80D00F08EF93D3966008400B74F949
:1035E2002FFF80C01F1F1F1F1FEF54FEF80303F79A
:1035F200E893FC08E893FD08E893FE08E893FF22AD
:1036020009E993C39D6008402974FB29F980F109F7
:10361200E993C39E6008401A74FA29F980E209E925
:1036220093D39F6008400B74F929F980D3191919B3
:103632001919E9C313C313FF22740093F8ECC3985A
:103642004024701F740193F8EDC3984019701474EC
:0E3652000293F8EEC398400E7009740393F8CB
:10366000EFC39840037F00227F0122EDF8E6F008C7
:10367000A3DFFA22EDF8E0F608A3DFFA22E0A36365
:10368000A201F0A363A201DFF475A20022E0A3630C
:10369000A201F0A363A201E0A363A201F0A363A2CD
:1036A00001E463A201F0A363A201DFE175A200229D
:1036B000E0A363A2016DFE936CFDEE058393FC1500
:1036C0008363A201DFEA75A200227F00E493A36373
:1036D000A201F00F600CA3E583C2E3F58363A201AE
:1036E00080EA75A20022E0A363A201F0A3E583C2F1
:1036F000E3F58363A201DFEE75A20022E0A363A2DB
:1037000001F0A3E583C2E4D2E3F58363A201DFEC19
:1037100075A20022E583C2E3F583E0A363A201F072
:10372000A363A201DFEE75A20022E583C2E4D2E327
:10373000F583E0A363A201F0A363A201DFEC75A20D
:103740000022F922C002C004C00612FFF0D006D049
:0437500004D002227D
:104D49000A536572763A00205544502054696D65BE
:104D59004750530A00200A444154414752414D3AB1
:104D690020002043414E2054696D654750530A0085
:104D790020547261737353656E644552520A002060
:104D89005265496E69742043414E0A002043414EE1
:104D9900283029203E20544F210A00205455203024
:094DA9000A0020545520310A00D3
:03001E00E4FF22DA
:10518D00C28DC2AF438901C28C906F56E0FF70078C
:10519D00F58A758CEE800AEFB40A06E4F58A758CF3
:0651AD0070D28CD2AF228B
:10515A00C28DC2AF438901C28C906F56E0FF7014B2
:10516A00302B09F58A758CDCC22B8012758A66751C
:10517A008CFC800AEFB40A06E4F58A758CDCD28CC2
:03518A00D2AF227F
:1051B300C22C906F56E0C394645006124DB2125144
:1051C3008D120022D22AE4F55790705EF0F545F572
:0651D3005BC22BF559221E
:10503900EF24FCF527200A127E4D7F4912436C7E2E
:105049006C7F2FE4FBAD27124603906C2EE0B41F52
:1050590003D22C22906C2F63A201906FDE63A20110
:0D506900AF2712367D852745E4F556C22895
:015076002217
:0F52C800D3EF6480948E5006E55B70028F5B22FB
:1024DA00208D030225E0C28C202A030226DDE55B5B
:1024EA0060519068B77D47FF123674E54764017002
:1024FA001E9068BFE0B4FF0ED22D200A127E4D7FD7
:10250A005012436C8009302D06E4F55B0226DD1279
:10251A00518D124E7A200A077E4D7F5E12436C203F
:10252A000A0B7E687FB7E4FBAD5B124603E4F55BFA
:10253A000226DDE545605C74E22556F582E4346FD7
:10254A00F583E02405F527D3940E4008E4F545D237
:10255A00280226DD74DE2556F582E4346FF5837D84
:10256A0047AF27123674E5272556F556E54730E773
:10257A0002D22BE547B40103202D0612518D124ECB
:10258A007AE556C3954550030226DDE4F545D2287F
:10259A000226DDE5586023906F427D47FF123674AC
:1025AA00E547B40109302D06E4F5580226DD12513B
:1025BA008D124E7AE4F5580226DD201016E55AC32C
:1025CA009464400320030C906F56E0C39464500354
:1025DA00124EDC12518D123D088F27EF700302262E
:1025EA00DD12515AE4F559E547B4010CD22D200AFF
:1025FA00077E4D7F6B12436CE55AC3946E4003020B
:10260A0026B42003030226B4302C75E547644270D1
:10261A006FE54B7032E549C454F0FFE54AC4540FE4
:10262A002FF547E54AC454F0F5487549087457250B
:10263A005AF582E4346FF5837403255AF55A7D47B7
:10264A007F0312366B80637457255AF582E4346F20
:10265A00F583E527255AF55A7D47AF2712366B30A1
:10266A000C48C3E55A9527FFE49400FE74572FF5EA
:10267A0082746F3EAF82FEE4FBAD27124603802AC6
:10268A00E547B4420DE54AB40208906B69E064017B
:10269A0060187457255AF582E4346FF583E52725C7
:1026AA005AF55A7D47AF2712366B300121E547208C
:1026BA00E71C906E2E7D47AF2712366BAF27124765
:1026CA0087EF700A200A077E4D7F7912436CAF2785
:1026DA00122B1C300D26906618E0C394FA5003E0C2
:1026EA0004F0300015906F56E0C39464500C0559FD
:1026FA00E55994F04004C2AF80FEC20D20020302E5
:10270A0027FEE5576031D39401400415578028907D
:10271A00705EE004F0E0D39403400D200A077E4D7A
:10272A007F8812436C1251B3200A077E4D7F95129F
:10273A00436CE4F557D22A302943E558703F906F2D
:10274A004204F0A37408F0A37480F0A37401F0A308
:10275A007406F0906FD9E0906F47F0906FDAE090CE
:10276A006F48F0906FDBE0906F49F0906FDCE0907B
:10277A006F4AF0E4A3F0A3F075580BC22930277210
:10278A00906FD7E07035E5587031906F427442F01F
:10279A00A37408F0906FD8E0906F44F0906FDDE07A
:1027AA00906F45F0A37401F0755806200A077E4D14
:1027BA007FA412436C906FD7E004F0906FD7E06467
:1027CA0002702FE558702B906F427402F0A37408C0
:1027DA00F0906FD8E0906F44F0A3F0A37401F07505
:1027EA005806200A077E4D7FAB12436C906FD7E0E4
:0727FA0004F0C202120026E8
:0128010022B4
:10507700E55A6037E4906D2BF0A3E55AF0906F2F57
:10508700E0906D2DF0302C06A3741FF08006906D14
:105097002E7419F0906F5763A201906D2F63A201D0
:0E50A700AF5A12367DE4F55A7F01227F0022B7
:0B52D700302805C2287F01227F002242
:0100210022BC
:0652FC00E4F55AF545221D
:0A52E200E49069BAF0A3F0A3F022F3
:105221002043616E457247495400200A00204361C2
:105231006E457272434821000A000A205265714589
:045241007272210064
:103D0800E59B541F6020200A1A7E527F2112436CC3
:103D1800E59B541FFF7E007D031245297E527F2BB1
:103D280012436CE4F59BE5BA30E010E4F5B375B1E5
:103D380080F5B2D22AF55790705EF0E5CFF47003A3
:103D4800023E39752901E4F528E5CFF455297003B9
:103D5800023E27E528C454F0F5B1E5B2547F64204B
:103D68006003023DF8E5B3540FF54B85BC47E5BD4C
:103D7800541FFF131313541FFFE5BD54E044184F9D
:103D8800F548E5BDC43354E0FFE5BE131313541FD3
:103D98004FF549E5BEC43354E0FFE5BF1313135490
:103DA8001F4FF54A85A34C85A34D85A34E85A34F88
:103DB80085A35085A35185A35285A353E4F5B2206A
:103DC800100CE547547EB5470575B350800375B3AD
:103DD800D0E54B700AE547547EB547037F00223093
:103DE8001008E54730E7037F0022E54B2405FF2252
:103DF800E5B2549F6023200A207E527F2E12436C26
:103E0800AFB27E007D03124529AFB37E007D031259
:103E180045297E527F3912436CE4F5B275B3D0E57B
:103E28002925E0F5290528E528C394085003023D13
:033E3800517F00B7
:013E3B002264
:104E7A00906F56E0C39464505675B180E4F5B3F56B
:104E8A00B28547BCE549C4135407FFE54854E04FCF
:104E9A00F5BDE54933333354F8FFE54AC4135407E3
:104EAA004FF5BEE54A33333354F8F5BF854CA38535
:104EBA004DA3854EA3854FA38550A38551A3855243
:104ECA00A38553A3E54B540F2450F5B375570AC273
:024EDA002A228A
:104EDC0075B190E5B220E613200A107E527F3B128A
:104EEC00436CAFB27E007D03124529E4F5B3F5B2F5
:104EFC00748D2516F582E43461F583E0F5BCE4F598
:104F0C00BD748E2516F582E43461F583E0FF3333EE
:104F1C003354F8F5BE75BF7805160516748D251635
:104F2C00F582E43461F583E07002F51675B3502216
:0952EC00EF6003C29622D2962263
:104DB20043AB01C2E8C2EAE4FFEFC454F0F5B1C369
:104DC200EF64809488500575B3D08003E4F5B3E4B2
:104DD200F5B2F5BCF5BDF5BEF5BFF5C4F5C5F5C632
:104DE200F5C7F5A3F5A3F5A3F5A3F5A3F5A3F5A3DD
:104DF200F5A30FBF0EC3906F56E0FF25E0F5B47523
:104E0200B50C75B66C75A11275AB0275C13E75C352
:044E1200FF75C20363
:014E16002279
:1033CE0000000000000000000000000000000000EF
:1033DE003FF3630041D5E80043B71B8045984F008B
:1033EE0047798280495C07804B3D3B004D1E6E80C5
:1033FE004EFFA20050E2270052C35A8054A48E0002
:10340E005685C180586846805A497A005C2AAD803C
:10341E005E0BE1005FEE660061CF998063B0CD0078
:10342E0065920080677485806955B9006B36EC80B3
:10343E006D1820006EFAA50070DBD8800000000029
:10344E000028DE80004DC8800076A700009E340064
:10345E0000C7123000EE9F8001177E0001405C8095
:10346E000167E9800190C80001B8550001E1338081
:10347E00000000000028DE80004F1A000077F88060
:10348E00009F858000C8640000EFF1000118CF8016
:10349E000141AE0001693B000192198001B9A6807D
:1034AE0001E2850000000000000151800002A3002F
:1034BE000003F48000054600000697800007E9002F
:1034CE0000093A80000A8C00000BDD80000D2F00F1
:1034DE00000E8080000FD2000011238000127500B4
:1034EE000013C68000151800001669800017BB0077
:1034FE0000190C80001A5E00001BAF80001D010039
:10350E00001E5280001FA4000020F58000224700FC
:10351E00002398800024EA0000263B8000278D00BF
:10352E000028DE800000000000000E1000001C20AD
:10353E0000002A3000003840000046500000546061
:10354E00000062700000708000007E9000008CA071
:10355E0000009AB00000A8C00000B6D00000C4E081
:10356E000000D2F00000E1000000EF100000FD208E
:10357E0000010B3000011940000127500001356099
:10358E0000014370000151801F1C1F1E1F1E1F1FB4
:04359E001E1F1E1FAF
:103F6500E55C25E025E024CEF582E43433F58312C3
:103F750029B28F658E648D638C62E55C540370286D
:103F8500E56125E025E0247AF582E43434F58312F1
:103F950029B2EF2565F565EE3564F564ED3563F514
:103FA50063EC3562F5628026E56125E025E024466F
:103FB500F582E43434F5831229B2EF2565F565EE13
:103FC5003564F564ED3563F563EC3562F562E55E00
:103FD50025E025E024AEF582E43434F5831229B2D8
:103FE500EF2565F565EE3564F564ED3563F563EC50
:103FF5003562F562E55FC3940C402AE56524C0F59A
:1040050065E56434A8F564E43563F563E43562F584
:1040150062E55F24F4FF7E007C0E7D10122848AA1D
:1040250006AB07800FAF5F7E007C0E7D101228481F
:10403500AA06AB07AE02E4FCFDE5652BF565E56474
:104045003EF564ED3563F563EC3562F562E5607563
:10405500F03CA4FFAEF0E4E5652FF565E5643EF5BB
:1040650064ED3563F563EC3562F562E4FEE56525DF
:104075005DF565EE3564F564ED3563F563EC356244
:02408500F562E2
:014087002216
:103BD300907076E0F55C25E025E024CEF582E434B0
:103BE30033F583E55CD3941F501DAF65AE64AD63BD
:103BF300AC6212363BEF700F74042582F582E43514
:103C030083F583055C80DC74FC2582F58274FF35C3
:103C130083F583AF821229C2C3E5659BF565E5642D
:103C23009AF564E56399F563E56298F562155CE5D9
:103C33005C14907076F0E55C5403700590347E80DC
:103C43000390344A7561307F617D621235A2A80406
:103C5300A905AA06C3E5659FF565E5649AF564E5DC
:103C63006399F563E56298F56205619034B2AF65D7
:103C7300AE64AD63AC627B007A00797C1236028F4E
:103C83005EEF25E025E024B2F582E43434F58312B7
:103C930029C2C3E5659BF565E5649AF564E5639917
:103CA300F563E56298F562055E903532AF65AE6403
:103CB300AD63AC627B007A00795C1236028F5FEFF2
:103CC30025E025E02432F582E43435F5831229C258
:103CD300C3E5659BF565E5649AF564E56399F5636A
:103CE300E56298F562AE64AF657C007D3C12285AAC
:103CF3008D5DAE64AF657C007D3C12285A8E648F67
:053D03006585656022EA
:101DBF0042415544004D415842005254530044454E
:101DCF004C4159005452414E5A0043414E004B5022
:101DDF0000544F52455000003E2A2C312CCFE0F0DA
:101DEF00E0ECE5F2F0FB20F3EFF0E0E2EBFFFEF9C1
:101DFF00E5E3EE20EAEEEDF2F0EEEBEBE5F0E020BE
:101E0F00CACF20C8F1E5F2FC0A003E4C2C6B3031F2
:101E1F002C25732C43EAEEF0EEF1F2FC20EDE020DE
:101E2F00F8E8EDE52043414E2C30202D20353030A1
:101E3F00EAE1283530EC292C31202D203530EAE12C
:101E4F0028353030EC290A0030202D20353030EA8B
:101E5F00E1283530EC290031202D203530EAE128FA
:101E6F00353030EC29003E532C6B30322C25627507
:101E7F002CCCE0EAF12E20E0E4F0E5F120E1EBEEEE
:101E8F00EAE020D2D128302D38290A003E532C6B9E
:101E9F0030332C2562752CCCE0EAF12E20E0E4F0F3
:101EAF00E5F120E1EBEEEAE020D2C8D228302D3860
:101EBF00290A003E532C6B30342C2562752CCCE054
:101ECF00EAF12E20E0E4F0E5F120E1EBEEEAE0208C
:101EDF00D2D328302D38290A003E422C6330312CC2
:101EEF002562752CC2F2EEF0E8F7EDFBE920EAEE81
:101EFF00EDF2F0EEEBEBE5F020EDE020F8E8EDE5AC
:101F0F000A003E2A2C312CCFE0F0E0ECE5F2F0FB9A
:101F1F0020EFF0EEF2EEEAEEEBE020CCDDCA203857
:101F2F0037302D352D31303120EFEE20EFEEF0F23E
:101F3F00F32052533233320A003E432C5061723138
:101F4F002C202562752CC0E4F0E5F1204153445557
:101F5F002028F4E8EAF1E8F0EEE2E0EDEDFBE92904
:101F6F000A003E432C506172322C20253034752FDD
:101F7F00253034752F253034752F253034752CCD01
:101F8F00E0F7E0EBFCEDFBE520E0E4F0E5F1E0202D
:101F9F00D2D12FD2C8D22FD2C8C82FD2D32028F453
:101FAF00E8EAF1E8F0EEE2E0EDEDFBE5290A003EAC
:101FBF004C2C6B30352C256C752CD1EAEEF0EEF1F4
:101FCF00F2FC20EEE1ECE5EDE020EDE020EFEEF0AD
:101FDF00F2F32C3130302C3230302C3330302C3671
:101FEF0030302C313230302C323430302C343830D9
:101FFF00302C393630302C31393230302C333834B4
:10200F0030302C35373630302C3131353230300AD4
:10201F00003E532C6B30362C2562752CCDEEECE543
:10202F00F0205254552028E82041534455290A00E6
:10203F003C21003C6B30313D003C6B30323D003C6D
:10204F006B30333D003C6B30343D003C6330313DF1
:10205F00003C6B30353D003C6B30363D00526573B4
:10206F007461727420424C0A0043414E2054552033
:10207F004F4B0A0043414E205455205265710A00C0
:10208F002054552054696D654F5554210A00204F37
:10209F004B2000204E414B200020526573204348B7
:1020AF000A2000205265732055500A200020444119
:1020BF005441410A200020545553656C0A200020DA
:1020CF005455455845430A200020444154410A20A5
:1020DF00002053657454696D650A200020434852EF
:1020EF000A2000205245510A20002054555F4F4BC3
:1020FF000A20002054555F4572720A200020545563
:10210F0052656164790A20002054555265616479E3
:10211F00320A200073656E642074730A0073656E53
:10212F00642074734379630A002073656E642074AE
:10213F0069744379630A20002073656E64207469A3
:10214F00690A20002073656E642074697453706F80
:10215F00740A2000FF1DBFFF1DC4FF1DC9FF1DCD49
:0F216F00FF1DD3FF1DD9FF1DDDFF1DE0FF1DE686
:03002300023E3C5E
:0B3E3C00C0E0C083C082C0D075D01869
:103E4700209803023F23C298756901AF9930130385
:103E5700023F5CD29120113CBFE507D21DD213026D
:103E67003F23BFA207D216D213023F23BF680DD24A
:103E770011D218750A00750E00023F23EF64106017
:103E870003023F23D211D219751502750E03750A65
:103E970000023F5CE50E70078F15050E023F5CE5DB
:103EA7000EB4010FE515B51F05050E023F5CC211E3
:103EB700023F5CE50EB4020AEF646860CEC21102ED
:103EC7003F5CE50EB4031E7471250FF582E434667A
:103ED700F583EFF0050F250AF50A1515E515707539
:103EE700750E048070E50EB4040DE50AB51F0405D0
:103EF7000E8062C211805EE50E6405701FBF161149
:103F0700D213850F15630F80530F80C211C29180A2
:103F170044C219C218530F80C21180393099363004
:103F2700123190618BE0FFE510C39F4008C212D2A7
:103F37001AC290801ED29074B12510F582E43467BE
:103F4700F583E0F513E50B5213A2D0B3929B8513CB
:053F5700990510C2995C
:093F5C00D0D0D082D083D0E03235
:10418C007BFF7A1D79E71221E0906F56E070147571
:10419C002FFF75301E7531577BFF7A1E791912214E
:1041AC00E08012752FFF75301E7531667BFF7A1E0D
:1041BC0079191221E07BFF7A1E797590618CE0F5FC
:1041CC002F1221E07BFF7A1E799B906101E0F52F85
:1041DC001221E07BFF7A1E79C2906100E0F52F126C
:1041EC0021E07BFF7A1E79E8A210E433F52F12212F
:1041FC00E07BFF7A1F79111221E07BFF7A1F79484F
:10420C00752F011221E07BFF7A1F797190640EE00B
:10421C00F52FA3E0F530906189E0F531A3E0F5329C
:10422C00906187E0F533A3E0F534906622E0F53534
:10423C00A3E0F5361221E09068B1E0FEA3E0FFC3E5
:10424C00E49FFFE49EFEAB07FA3395E0F9F87F009C
:10425C007E8C7D0A7C001229018F328E318D308C40
:10426C002F7BFF7A1F79BE1221E07BFF7A20792009
:0A427C0090640DE0F52F1221E022FE
:10444D007E207F3F124953EF4E70037F0122E4908F
:10445D006F56F07E207F42124953EF4E6015125277
:10446D007EBF3106906F56740AF0BF3206906F56BC
:10447D007464F07E207F48124953EF4E6008124F4E
:10448D003C90618CEFF07E207F4E124953EF4E60D1
:10449D0008124F3C906101EFF07E207F541249537A
:1044AD00EF4E6008124F3C906100EFF07E207F5A76
:1044BD00124953EF4E600D124F3CEC4D4E4F24FF01
:1044CD0092108002C2107E207F60124953EF4E6021
:1044DD0023124F3CA804A905AA06AB077F007E8CCA
:1044ED007D0A7C001229011229939068B1EEF0A388
:1044FD00EFF0800A9068B174FFF0A374DCF07E20B9
:10450D007F66124953EF4E600A124F3C90640DEFD7
:0B451D00F0800690640D7401F07F0038
:014528002270
:102FDF00E490640DF0906F56F090706EF090706EFC
:102FEF00E075F003A42463F582E43421F583E493C0
:102FFF00FB740193FA740293F912280270030231E1
:10300F00DAE4907070F0A3F090706FF090706FE052
:10301F0024E2F582E43469F583E0FF70030231D1D5
:10302F0090706EE075F003A42463F582E43421F50B
:10303F0083E493FB740193FA740293F9907070E038
:10304F00F58275830012281BFEEFB5060F90707185
:10305F007401F0907070E004F00231C8907071E06C
:10306F0070030231C8EE60030231BF90706EE0B49E
:10307F00070040030231D190308DF82828730230B9
:10308F00A20230EF02312C0231310230A202315F45
:10309F0002318F90706FE024E2F9E43469FA7B011A
:1030AF00C0031B8B2F753000753100E4F532D00350
:1030BF001237549070721229D2907072E0F8A3E018
:1030CF00F9A3E0FAA3E0FB7F007E8C7D0A7C00125F
:1030DF0029011229939068B1EEF0A3EFF00231D1DC
:1030EF0090706FE0FD24E2F582E43469F583E0240B
:1030FF00D090618CF074E32DF582E43469F583E0B0
:10310F0024D0906101F090706FE024E4F582E434F4
:10311F0069F583E024D0906100F00231D1D217021B
:10312F0031D190706FE024E2F9E43469FA7B01C089
:10313F00031B8B2F753000753100E4F532D003126D
:10314F0037549070721229D2907075E0F509807221
:10315F0090706FE024E2F9E43469FA7B01C0031B3D
:10316F008B2F753000753100E4F532D003123754D0
:10317F009070721229D2907075E0906F56F0804265
:10318F0090706FE024E2F9E43469FA7B01C0031B0D
:10319F008B2F753000753100E4F532D003123754A0
:1031AF009070721229D2907075E090640DF08012B9
:1031BF00E4907071F0907070F090706FE004F00216
:0B31CF00301B90706EE004F0022FEC4B
:0131DA0022D2
:102DD0009069B8E064557004A3E064816064E4F530
:102DE0001074192510F582E43466F583E4F074104C
:102DF0002510F582E43466F583E4F074052510F5BA
:102E000082E43463F583E4F00510E510B408D2E4FD
:102E1000F51074712510F582E43467F583E4F0054C
:102E200010E510B440ECE4F51074BD2510F582E413
:102E30003461F583E4F00510E510B480ECE4F5129C
:102E4000F511E4907076F0C212C21AC211C213F5E5
:102E50001090618BF0F509F508F50FF569C20FC206
:102E60001CC2179068B174FFF0A374F4F0750BFFE7
:102E70009061007402F0A3F090618CF090640EE415
:102E8000F0A304F09061897403F0A374E9F09061F9
:102E900087740BF0A374B9F09066227407F0A374E2
:102EA000D1F012444DEF6003122FDFE4F51690705D
:102EB0006C7461F0A3748DF090618CE0F516E516EA
:102EC000C394014007E516D394084003E4F516E5E2
:102ED00016602890706CE475F0011228AF85F082BE
:102EE000F58374C4F0151690706CE475F001122827
:102EF000AF85F082F583E516F080D4906101E0F5AE
:102F000016E516C394014007E516D394084003E480
:102F1000F516E516602890706CE475F0011228AF84
:102F200085F082F58374C8F0151690706CE475F026
:102F3000011228AF85F082F583E516F080D4906108
:102F400000E0F516E516C394014007E516D3940892
:102F50004003E4F516E516602890706CE475F00106
:102F60001228AF85F082F58374C2F0151690706C4C
:102F7000E475F0011228AF85F082F583E516F08044
:102F8000D490706CE475F0011228AF85F082F5835F
:102F9000E4F090706C75F0011228AF85F082F58333
:102FA000E4F0F516C291C290C2ADF5C9D2CDD2CC33
:102FB000C2C9C2CAF5CDF5CC9068B1E0F5CBA3E0AB
:102FC000F5CA85CBCD85CACCD29FD29ED29CD2CA1F
:0E2FD000C2ACC298C29975B81075B710D2ACD9
:012FDE0022D0
:0246D7008F2D25
:1046D900E4FF7C617D02FEEEC3952D50120DEDAA1B
:1046E9000470010C14F5828A83E02FFF0E80E80D17
:1046F900EDAA0470010C14F5828A83EFF00DEDAE7A
:104709000470010C14F5828E837416F0052D052DA5
:104719007E677FB17C617D02E52DB4040E8F828EA8
:10472900837410F00FBF00010E80328F828E837464
:1047390068F00FBF00010EE52D24FEFB8F828E83EA
:10474900F00FBF00010E8F828E83EBF00FBF0001C7
:104759000E8F828E837468F00FBF00010E8C838DDB
:104769008263A2018E838F8263A201AF2D12367DEF
:0D477900E52DB4040304FF22E52D2404FF08
:014786002210
:1050B5002012351246D790618BEFF0200A0B7E67E0
:1050C5007FB1E0FDE4FB1246033017057F01125264
:1050D500ECE5096003F56622E4906618F0F510D258
:0950E50012C2992099FDD2992212
:022B1C008F2800
:102B1E0090640DE07003022DCFE54730E712E54AD1
:102B2E00B4100D200A077E207F6C12436CE4F5086A
:102B3E00E54724BE7003022D9C24FA7003022CC4B8
:102B4E0024046003022DCFE54830E703022BEDE5A8
:102B5E004A6066E549C394024003022DCFE54970F1
:102B6E0007E54A14F5298006E54A241FF529E529CB
:102B7E0075F004A4240DF582746335F0F5837D4C55
:102B8E007F0412366BE52975F004A42405F58274D2
:102B9E006235F0F5837D507F0412366B74FD254946
:102BAE00F582E43461F5837481F074BD2529F582D4
:102BBE00E43461F5837401F02274102549F582E442
:102BCE003466F583E04480F0E54925E025E02445B0
:102BDE00F582E43466F5837D4C7F0412366B22E574
:102BEE004B64086003022DCF752801E54A5407FF98
:102BFE00E528A807088002C333D8FCF528740825F9
:102C0E0012F512B5110674082511F511E54A547F17
:102C1E00FFE549C43354E02FFE74002512F582E41B
:102C2E003460F583EEF0E54AC39480503CEF131305
:102C3E0013541FFFE54925E025E025E025E0244556
:102C4E00F582E43466F583E5822FF582E43583F56B
:102C5E0083E0FFE528F4FEEF5EF074012512F582A5
:102C6E00E43460F583E4F0803AE54A547FFF1313B1
:102C7E0013541FFFE54925E025E025E025E0244516
:102C8E00F582E43466F583E5822FF582E43583F52B
:102C9E0083E04528F074012512F582E43460F58353
:102CAE007401F074022512F582E43460F5837D4CD4
:102CBE007F0612366B22E54A54E06440702CE54ADA
:102CCE00540F144440FF74052549F582E43463F52E
:102CDE0083EFF0E54925E025E02424F582E434660F
:102CEE00F5837D4C7F0412366B2274052549F582DF
:102CFE00E43463F583E0F56030E64AE54A13135495
:102D0E003FFFE560540FB50714E56054074480FF9C
:102D1E0074052549F582E43463F583EFF0E54A54F2
:102D2E007FFF1313543FFF75F008E549A42FF5827A
:102D3E00E435F0F583E5822471F582E5833467F599
:102D4E0083E4F08027E54A547FFF1313543FFF7549
:102D5E00F008E549A42FF582E435F0F583E58224E9
:102D6E0071F582E5833467F5837401F075F040E503
:102D7E0049A42410F582E5F03464F583E54A547FC6
:102D8E0075F002122A0F7D4CAF4B12366B22302794
:102D9E0030E54AB40112200A077E207F7812436C78
:102DAE00E54D0490705FF022E54AB40314906FD79E
:102DBE00E0B401037405F0200A077E207F831243DE
:012DCE006C98
:012DCF0022E1
:1000260030001DC200302718906184E004F0E0D350
:100036009414400C200A077E207F8F12436CC2273F
:10004600E5147036906644E004F0E05407F0E0FFF3
:100056002405F582E43463F583E0FE30E71C74057D
:100066002FF582E43463F583EE547FF074052FF5A3
:1000760082E43463F583E004F514201B2690618541
:10008600E004F0E0543FF0E0FF2471F582E43467C9
:10009600F583E0600ED21B74712FF582E43467F5A8
:1000A60083E4F0201426906621E004F0E0543FF04B
:1000B600E0FF24BDF582E43461F583E0600ED214DE
:1000C60074BD2FF582E43461F583E4F020152A909F
:1000D6006186E004F0E05407F0E0FF2410F582E4C6
:1000E6003466F583E0FE30E71074102FF582E434B1
:1000F60066F583EE547FF0D215201303020A17E546
:100106001554802471F582E43466AF82F5298F2A6E
:10011600301D0CC21D200A077E207F9D12436C30C5
:10012600160CC216200A077E207FA212436C2018E6
:1001360006201903020A15852A82852983A3E0FF72
:1001460090640DE0FEEF6E6003020A11E52A2407B3
:10015600F582E43529F583E0FEE52A2406F582E4F6
:100166003529F583E07C002400F52CEC3EF52B8543
:100176002A82852983E0544F24BF603E24FE6054C2
:100186001470030202B924FB7003020416147003F0
:10019600020436147003020436240B6003020A11AB
:1001A600200A077E207FA812436CE50B54E5F5284C
:1001B600A2D0929B7599E5020A11200A077E207F3C
:1001C600B212436CE50B54E5F528A2D0929B7599C3
:1001D600E5020A11200A077E207FBC12436CE50B5C
:1001E60054E5F528A2D0929B7599E5852A82852942
:1001F60083A3A3E0642D6003020A11852983852A5F
:100206008263A20190666563A2017F0A12367DE5CC
:100216002A2404F582E43529F583E0543F64066018
:10022600030202B4E52A2408F582E43529F583E0C1
:1002360030E75A200A077E207FC512436C30270319
:10024600020A11D227E4906FD7F0906184F090668D
:1002560022E0FEA3E0FFC3E52C9FFDE52B9EC4F83C
:1002660054F0C868EDC4540F48906FD8F0ED540FA1
:1002760025E0FFE433E52A2408F582E43529F583F1
:10028600E0640154012F906FDDF0020A11200A0785
:100296007E207FCE12436C202703020A11906FD76F
:1002A600E064066003020A117402F0020A11C22712
:1002B600020A11200A077E207FD812436C852A8203
:1002C600852983A3A3E06467600302036F200A07FE
:1002D6007E207FE012436C75080AE52A2408F58221
:1002E600E43529F583E0750C00F50DE52A2409F5BA
:1002F60082E43529F583E0FEE4EE420CE52A240A81
:10030600F582E43529F583E0F560E52A240BF582CC
:10031600E43529F583E0F55FE52A240CF582E4351A
:1003260029F583E0F55EE52A240DF582E43529F505
:1003360083E0F561E52A240EF582E43529F583E0AC
:10034600F55CAE0CAF0D7C037DE812285A8F5D126A
:100356003F65906FD9E565F0A3E564F0A3E563F02A
:10036600A3E562F0D229020A11852A82852983A390
:10037600A3E0642D6003020A11852983852A82631E
:10038600A20190666563A2017F0A12367DE52A24E2
:1003960004F582E43529F583E0543F6406706CE584
:1003A6002A2408F582E43529F583E0FD30E7453057
:1003B6002703020A11D227E4906FD7F090705FF0FE
:1003C600906622E0FEA3E0FFC3E52C9FFBE52B9E93
:1003D600C4F854F0C868EBC4540F48906FD8F0EBDB
:1003E600540F25E0FFE433ED640154012F906FDDD7
:1003F600F0020A11202703020A11906FD7E0640663
:100406006003020A117402F0020A11C227020A11DD
:10041600200A077E207FEB12436C906102740BF07A
:1004260090640DE0906103F07F021250B5020A114C
:10043600200A077E207FF212436CE508C39405501C
:10044600050508020A1120270302053990705FE0AE
:10045600FF60686401702E200A077E207FF9124330
:100466006C90666563A20190610263A2017F091226
:10047600367D9061027408F0906106740AF07F0977
:100486001250B5802C200A077E217F0212436C9001
:10049600666563A20190610263A2017F0912367D3F
:1004A6009061027408F09061067447F07F0912505B
:1004B600B5E490705FF0C227020A11906FD7E0642E
:1004C600057034200A077E217F0C12436C90666506
:1004D60063A20190610263A2017F0912367D9061D9
:1004E600027408F090610614F07F091250B5906FFF
:1004F600D77406F0020A11906FD7E06403703420B7
:100506000A077E217F1712436C90666563A20190ED
:10051600610263A2017F0912367D9061027408F0C0
:1005260090610614F07F091250B5906FD77407F0EA
:10053600020A11E51265117003020627E511240867
:10054600F52874082511F511D21C9061027408F083
:1005560090640DE0906103F0A3741EF0A37401F0A3
:10056600A37403F0A37401F090640FE0FF740025F8
:1005760028F582E43460F583E0FE2F906108F0EE02
:10058600FF90640FE02F90640EE03400FF3395E097
:10059600906109EFF074012528F582E43460F58353
:1005A600E090610AF074022528F582E43460F58350
:1005B600E0F56574032528F582E43460F583E0F5FB
:1005C6006474042528F582E43460F583E0F56374E9
:1005D600052528F582E43460F583E0F562123BD305
:1005E600AF5D7E007C037DE81228488E0C8F0DEFF0
:1005F60090610BF0E50CA3F0A3E560F0A3E55FF0D6
:10060600A3E55EF0A3E561F0A3E55CF07F10125070
:10061600B5300A03020A117E217F2312436C020AB7
:10062600112015030206E1C2159061027408F090CC
:10063600640DE0906103F0A37407F0A37401F0A3C6
:10064600F0A3F090640FE0FF906186E0FEC433549F
:10065600E02F906108F0EE75F020A4FF90640FE0A3
:100666002F90640EE035F0FF3395E0906109EFF0CE
:10067600906186E0FF25E025E02445F582E43466B6
:10068600F583E090610AF0EF25E025E02446F58247
:10069600E43466F583E090610BF0906186E025E036
:1006A60025E02447F582E43466F583E090610CF09A
:1006B600EF25E025E02448F582E43466F583E090F2
:1006C600610DF0E4A3F07F0D1250B5300A03020A63
:1006D600117E217F2C12436C020A11E5147003026D
:1006E6000851200A077E217F3812436CE51425E065
:1006F60025E0F560E4F5149061027408F090640D4D
:10070600E0906103F0A37422F0E5602480A3F0A3D7
:100716007401F0A3F090618AE0FF906644E0FEC4A5
:100726003354E02F906108F0EE75F020A4FF90613D
:100736008AE02F906189E035F0FF3395E0906109FA
:10074600EFF0906644E075F040A42410F582E5F0E1
:100756003464F58363A20190610A63A201AF60125B
:10076600368DE56075F003A42408F528906644E00C
:10077600FF25E025E02424F582E43466F583E0F5E0
:1007860065EF25E025E02425F582E43466F583E06F
:10079600F564906644E0FF25E025E02426F582E432
:1007A6003466F583E0F563EF25E025E02427F5823E
:1007B600E43466F583E0F562123BD3AF5D7E007CE0
:1007C600037DE81228488E0C8F0DEFAE280528749D
:1007D600022EF582E43461F583EFF0E50CFFAE28D6
:1007E600052874022EF582E43461F583EFF0AF2814
:1007F600052874022FF582E43461F583E560F0AFD5
:1008060028052874022FF582E43461F583E55FF04C
:10081600AF28052874022FF582E43461F583E55E7E
:10082600F0AF28052874022FF582E43461F583E5DC
:1008360061F0AF28052874022FF582E43461F58350
:10084600E55CF0AF281250B5020A11201403020924
:100856007A200A077E217F4712436CC214906102F8
:100866007408F090640DE0906103F0A37425F0A382
:100876007401F0A3F0A3F0906188E0FF906621E098
:10088600FE2F906108F0EEFF906188E02F9061875F
:10089600E03400FF3395E0906109EFF0906621E0C7
:1008A60025E025E0F528FF0528740D2FF582E434B0
:1008B60063F583E090610AF0AF280528740D2FF5E3
:1008C60082E43463F583E090610BF0AF2805287469
:1008D6000D2FF582E43463F583E090610CF0AF28C8
:1008E6000528740D2FF582E43463F583E090610DDD
:1008F600F0E4A3F074FC2528F528FF052874052FDD
:10090600F582E43462F583E0F565AF2805287405C1
:100916002FF582E43462F583E0F564AF2805287488
:10092600052FF582E43462F583E0F563AF280528E8
:1009360074052FF582E43462F583E0F562123BD349
:10094600AF5D7E007C037DE81228488E0C8F0DEF8C
:1009560090610FF0E50CA3F0A3E560F0A3E55FF06E
:10096600A3E55EF0A3E561F0A3E55CF07F14125009
:10097600B5020A11201B030209FE200A077E217F09
:100986005312436CC21B9061027408F090640DE030
:10099600906103F0A37409F0A37484F0A37403F0C8
:1009A600A37401F090618AE0FF906185E0FE25E086
:1009B60025E02F906108F0EE75F004A4FF90618A9F
:1009C600E02F906189E035F0FF3395E0906109EF03
:1009D600F0906185E075F008A42410F582E5F03406
:1009E60064F58363A20190610A63A2017F04123653
:1009F6008D7F141250B580139061027409F09064D3
:100A06000DE0906103F07F021250B5C219C218C200
:010A160013CC
:010A170022BC
:0100220022BB
:1048D30002125BE493A3F8E493A34003F68001F28E
:1048E30008DFF48029E493A3F85407240CC8C333E6
:1048F300C4540F4420C8834004F456800146F6DFB5
:10490300E4800B01020408102040809052F5E47EFD
:10491300019360BCA3FF543F30E509541FFEE493A9
:10492300A360010ECF54C025E060A840B8E493A370
:10493300FAE493A3F8E493A3C8C582C8CAC583CA9B
:10494300F0A3C8C582C8CAC583CADFE9DEE780BE53
:0152FB0000B2
:10280200BB010689828A83E0225002E722BBFE02D4
:09281200E32289828A83E4932207
:10281B00BB010CE58229F582E5833AF583E0225072
:10282B0006E92582F8E622BBFE06E92582F8E222BC
:0D283B00E58229F582E5833AF583E49322D6
:10284800EF8DF0A4A8F0CF8CF0A428CE8DF0A42EA4
:02285800FE225E
:10285A00BC000BBE0029EF8DF084FFADF022E4CC62
:10286A00F875F008EF2FFFEE33FEEC33FCEE9DEC2B
:10287A00984005FCEE9DFE0FD5F0E9E4CEFD22ED71
:10288A00F8F5F0EE8420D21CFEADF075F008EF2FBB
:10289A00FFED33FD4007985006D5F0F222C398FDAC
:0528AA000FD5F0EA2249
:1028AF00A3F8E0C5F025F0F0E582158270021583DC
:0628BF00E0C838F0E82239
:1028C50075F008758200EF2FFFEE33FECD33CDCCCA
:1028D50033CCC58233C5829BED9AEC99E58298404D
:1028E5000CF582EE9BFEED9AFDEC99FC0FD5F0D62A
:1028F500E4CEFBE4CDFAE4CCF9A88222B800C1B954
:102905000059BA002DEC8BF084CFCECDFCE5F0CB91
:10291500F97818EF2FFFEE33FEED33FDEC33FCEBCA
:1029250033FB10D703994004EB99FB0FD8E5E4F985
:10293500FA227818EF2FFFEE33FEED33FDEC33FC72
:10294500C933C910D7059BE99A4007EC9BFCE99A66
:10295500F90FD8E0E4C9FAE4CCFB2275F010EF2FAB
:10296500FFEE33FEED33FDCC33CCC833C810D707AB
:102975009BEC9AE899400AED9BFDEC9AFCE899F8E6
:0E2985000FD5F0DAE4CDFBE4CCFAE4C8F92279
:0E299300C3E49FFFE49EFEE49DFDE49CFC2255
:1029A100EB9FF5F0EA9E42F0E99D42F0E89C45F08C
:0129B1002203
:1029B200E493FC740193FD740293FE740393FF226B
:1029C200E493F8740193F9740293FA740393FB226B
:0C29D200ECF0A3EDF0A3EEF0A3EFF02278
:1029DE00A8828583F0D083D0821229F51229F512B0
:1029EE0029F51229F5E473E493A3C583C5F0C583D5
:1029FE00C8C582C8F0A3C583C5F0C583C8C582C843
:012A0E0022A5
:0C2A0F00A42582F582E5F03583F58322D2
:10217E00E53B242FF8E6053B22782C302502782FFC
:10218E00E475F001122A7C022802201EEB7F2ED26B
:10219E001E8018EF540F2490D43440D4FF30220BFD
:1021AE00EF24BFB41A0050032461FFE53C60021512
:1021BE003C053FE53F7002053E30250D782CE47559
:1021CE00F001122A7CEF022A1B024FF27403D22571
:1021DE008003E4C225F53B8B2C8A2D892EE4F53C39
:1021EE00F53EF53FE53C60077F201221B980F5757D
:1021FE003DFFC21FC21EC220C221C223C224C2265C
:10220E00122187FF700D3025057F001221CAAF3FC6
:10221E00AE3E22B4255FC2D5C222122187FF24D042
:10222E00B40A00501A75F00A783C30D50508B6FF8E
:10223E000106C6A426F620D5047002D22180D92428
:10224E00CFB41A00EF5004C2E5D2220223CAD21F25
:10225E0080C6D21E80C0D22080BCD2D580BAD223F6
:10226E0080B47F201221B92020077401B53C0040B4
:10227E00F112217EFF1221B90221F2D226D2248040
:10228E009512217EFB12217EFA12217EF94A4B70A5
:10229E0006799B7A247BFF20202EE53C602A7E0067
:1022AE008E8275830012281B60060EEE653D70F05F
:1022BE00C2D5EBC0E0EAC0E0E9C0E0EE122411D0D6
:1022CE00E0F9D0E0FAD0E0FB122802FF60AAEBC0E2
:1022DE00E0EAC0E0E9C0E01221B9D0E02401F9D073
:1022EE00E03400FAD0E0FBE53D0460DCD53DD9805A
:1022FE00877BFF7A24790DD220809C791080027919
:10230E0008C224C2268008D2D5790A8004790AC26E
:10231E00D5E53D047002F53DE4FAFDFEFF12217E87
:10232E00FC7B08201F1312217EFD7B10301E0A122B
:10233E00217EFE12217EFF7B20EC3382D592D5507A
:10234E0013C3E4301E069FFFE49EFEE4201F039D90
:10235E00FDE49CFCE4CBF8C21FEC700CCFCECDCCD0
:10236E00E824F8F870F38017C3EF33FFEE33FEED79
:10237E0033FDEC33FCEB33FB994002FB0FD8E9EB5A
:10238E00301F05F8D0E0C448B21FC0E00AEC4D4E35
:10239E004F78207B0070C2EAB53D0040BCC0E01211
:1023AE002413D0F0D0E0201F04C4C0E0C4B21FC07C
:1023BE00F01221A2D0F0D5F0EB0221F2122ADB228C
:1023CE008F5323095822604C225C42230D4F231554
:0F23DE0044231549227543231B5522FF4622FF36
:1023ED004522FF4724BB5022642D22682E228B2BC1
:1023FD00226C2322892024A42A222448000022832F
:10240D003F3F3F00790AA2D5202114302309B9108E
:10241D00020404B9080104A2D520240250010420AD
:10242D0020689220B53C005034C0E07F2030211947
:10243D007F30A22072247223500F12246AC220C250
:10244D0024C223C2267F30800F302303E9C0E0125F
:10245D0021B9302303D0E0F9D0E0B53CCC302317BF
:10246D007F30B9100C1221B97F583022077F788048
:10247D0003B908031221B93020057F2D0221B97F40
:10248D00202026F87F2B2024F322922080CF286E47
:10249D00756C6C2900D21F12217E301FF8C21F7877
:1024AD003C30D50108F60222242D50434958122103
:1024BD007E2403B405004001E49024B6931221AAB2
:0D24CD00743A1221AAD221753C04022309A1
:103754008B2C8A2D892EE4F538F537F536F535F5B9
:1037640033F534E5304531452F6012EBC0E0EAC053
:10377400E0E9C0E0AB2FAA30A931122A8CAB2C05AA
:103784002EE52EAA2D7002052D14F9122802F53902
:10379400C394094007E539D3940D40E1E539642029
:1037A40060DBE539B42D054334038016E539B42BC9
:1037B40005433401800C74FF252EF52E74FF352D3E
:1037C400F52DE53260046410703FAB2CAA2DA92EB0
:1037D40012280264306009E532702E75320A80299D
:1037E40090000112281BFF64786004EFB45813435F
:1037F40034017532107402252EF52EE4352DF52D85
:103804008007E5327003753208AB2C052EE52EAA2D
:103814002D7002052D14F9122802F539C394614064
:103824000AE539D3947A50035339DF74D02539F536
:1038340039C3940A400CE5399411406D74F9253963
:10384400F539E539D39532506043340185383D85E7
:10385400373C85363B85353AAF327E00E4FCFDAB20
:1038640038AA37A936A835122A2DC8ECC8C9EDC91B
:10387400CAEECACBEFCBE4FCFDFEEB2539F538EEFE
:103884003AF537ED39F536EC38F535AF38AE37ADB6
:1038940036FCAB3DAA3CA93BA83AD31229A150035C
:1038A40002380D43340402380DE53420E003E4808B
:1038B4002DE5304531452F601EAB2CE52E24FFF954
:1038C400E52D34FFFAEBC0E0EAC0E0E9C0E0AB2F3D
:1038D400AA30A931122A8CE53430E20774FFFFFEC6
:1038E400FDFC22E534AF38AE37AD36AC3530E103FC
:0438F40002299322F0
:102A1B00BB010689828A83F0225002F722BBFE019A
:022A2B00F32294
:102A2D00E88FF0A4CC8BF0A42CFCE98EF0A42CFC48
:102A3D008AF0EDA42CFCEA8EF0A4CDA8F08BF0A4C6
:102A4D002DCC3825F0FDE98FF0A42CCD35F0FCEB25
:102A5D008EF0A4FEA9F0EB8FF0A4CFC5F02ECD39EA
:0F2A6D00FEE43CFCEAA42DCE35F0FDE43CFC2257
:102A7C00FAE6FB0808E6F925F0F618E6CA3AF6225B
:102A8C00BB011A89828A83D0F0D0E0F8D0E0F9D06B
:102A9C00E0FAD0E0FBE8C0E0C0F0022B0A5016E9E7
:102AAC00F8D083D082D0E0F9D0E0FAD0E0FBC0823D
:102ABC00C083022B01BBFE16E9F8D083D082D0E094
:0F2ACC00F9D0E0FAD0E0FBC082C083022B1322C6
:102ADB00D083D082F8E4937012740193700DA3A38A
:102AEB0093F8740193F5828883E47374029368609E
:062AFB00EFA3A3A380DF9E
:092B0100EBF608EAF608E9F622F9
:092B0A00EBF0A3EAF0A3E9F022CC
:092B1300EBF208EAF208E9F222F3
:00000001FF
